** EXPERIMENTAL (HLL) ** Open Watcom Linker Version 1.6beta1 Limited Availability
Portions Copyright (c) 1985-2002 Sybase, Inc. All Rights Reserved.
Created on:       13/11/17 16:24:33
Warning! W1121: file U:/tmp\ldconv__iomodule_obj_18eb52885a171700f8.obj(U:\DEV\python-2.7.5\Modules\_io\_iomodule.c): '_init_io' has already been exported
Executable Image: build/lib.os2knix-2.7/_io.pyd
creating an OS/2 EMX dynamic link library


                        +------------+
                        |   Groups   |
                        +------------+

Group                           Address              Size
=====                           =======              ====

CGROUP                          0001:00000000        00010fa0
DGROUP                          0002:00000000        000073a0



                        +--------------+
                        |   Segments   |
                        +--------------+

Segment                Class          Group          Address         Size
=======                =====          =====          =======         ====

TEXT32                 CODE           CGROUP         0001:00000000   00010fa0
________TEXT           CODE           CGROUP         0001:00010fa0   00000000
DATA32                 DATA           DGROUP         0002:00000000   00007160
SET1__os2dll           DATA           DGROUP         0002:00007160   00000004
SET2__os2dll           DATA           DGROUP         0002:00007164   00000000
SET3__os2dll           DATA           DGROUP         0002:00007164   00000004
SET1___CTOR_LIST__     DATA           DGROUP         0002:00007168   00000004
SET2___CTOR_LIST__     DATA           DGROUP         0002:0000716c   00000000
SET3___CTOR_LIST__     DATA           DGROUP         0002:0000716c   00000004
SET1___DTOR_LIST__     DATA           DGROUP         0002:00007170   00000004
SET2___DTOR_LIST__     DATA           DGROUP         0002:00007174   00000000
SET3___DTOR_LIST__     DATA           DGROUP         0002:00007174   00000004
SET1___crtinit1__      DATA           DGROUP         0002:00007178   00000004
SET2___crtinit1__      DATA           DGROUP         0002:0000717c   00000000
SET3___crtinit1__      DATA           DGROUP         0002:0000717c   00000004
SET1___crtexit1__      DATA           DGROUP         0002:00007180   00000004
SET2___crtexit1__      DATA           DGROUP         0002:00007184   00000000
SET3___crtexit1__      DATA           DGROUP         0002:00007184   00000004
SET1___eh_frame__      DATA           DGROUP         0002:00007188   00000004
SET2___eh_frame__      DATA           DGROUP         0002:0000718c   00000008
SET3___eh_frame__      DATA           DGROUP         0002:00007194   00000004
SET1___eh_init__       DATA           DGROUP         0002:00007198   00000004
SET2___eh_init__       DATA           DGROUP         0002:0000719c   00000004
SET3___eh_init__       DATA           DGROUP         0002:000071a0   00000004
SET1___eh_term__       DATA           DGROUP         0002:000071a4   00000004
SET2___eh_term__       DATA           DGROUP         0002:000071a8   00000004
SET3___eh_term__       DATA           DGROUP         0002:000071ac   00000004
SET1___fork_parent1__  DATA           DGROUP         0002:000071b0   00000004
SET2___fork_parent1__  DATA           DGROUP         0002:000071b4   00000000
SET3___fork_parent1__  DATA           DGROUP         0002:000071b4   00000004
SET1___fork_child1__   DATA           DGROUP         0002:000071b8   00000004
SET2___fork_child1__   DATA           DGROUP         0002:000071bc   00000000
SET3___fork_child1__   DATA           DGROUP         0002:000071bc   00000004
________DATA           DATA           DGROUP         0002:000071c0   00000000
BSS32                  BSS            DGROUP         0002:000071c0   00000040
c_common               BSS            DGROUP         0002:00007200   000001a0
________BSS            BSS            DGROUP         0002:000073a0   00000000


                        +----------------+
                        |   Memory Map   |
                        +----------------+

* = unreferenced symbol
+ = symbol only referenced locally

Address        Symbol
=======        ======

Module: U:\usr\lib\dll0hi.obj({standard input})
0001:00000000* __text
0002:00000000* __data
0002:00000000* ___data_start
0002:000071c0* ___bss_start
0002:00007160+ __os2dll
0002:00007168  ___CTOR_LIST__
0002:00007170  ___DTOR_LIST__
0002:00007178* ___crtinit1__
0002:00007180* ___crtexit1__
0002:00007188  ___eh_frame__
0002:00007198  ___eh_init__
0002:000071a4  ___eh_term__
0002:000071b0+ ___fork_parent1__
0002:000071b8+ ___fork_child1__
Module: U:/tmp\ldconv_bufferedio_obj_18eb52885a17165130.obj(U:\DEV\python-2.7.5\Modules\_io\bufferedio.c)
0001:00004cf5  __PyIO_trap_eintr
0002:000002c0  _PyBufferedReader_Type
0002:000001f0  _PyBufferedWriter_Type
0002:00000050  _PyBufferedRandom_Type
0002:00000120  _PyBufferedRWPair_Type
0002:00000390  _PyBufferedIOBase_Type
Module: U:/tmp\ldconv_bytesio_obj_18eb52885a17168010.obj(U:\DEV\python-2.7.5\Modules\_io\bytesio.c)
0002:000014b0  _PyBytesIO_Type
Module: U:/tmp\ldconv_fileio_obj_18eb52885a1716a720.obj(U:\DEV\python-2.7.5\Modules\_io\fileio.c)
0001:00007a71  __PyFileIO_closed
0002:000020e0  _PyFileIO_Type
Module: U:/tmp\ldconv_iobase_obj_18eb52885a1716ce30.obj(U:\DEV\python-2.7.5\Modules\_io\iobase.c)
0001:00008434  __PyIOBase_check_writable
0001:000084dc  __PyIOBase_check_readable
0001:00008584  __PyIOBase_check_seekable
0001:000088ad  __PyIOBase_check_closed
0001:00008a6b  __PyIOBase_finalize
0002:00002be0  _PyRawIOBase_Type
0002:00002cb0  _PyIOBase_Type
Module: U:/tmp\ldconv__iomodule_obj_18eb52885a171700f8.obj(U:\DEV\python-2.7.5\Modules\_io\_iomodule.c)
0002:00007200  __PyIO_str_close
0002:00007210  __PyIO_str_closed
0002:00007220  __PyIO_str_decode
0002:00007230  __PyIO_str_encode
0002:00007240  __PyIO_str_fileno
0002:00007250  __PyIO_str_flush
0002:00007260  __PyIO_str_getstate
0002:00007270  __PyIO_str_isatty
0002:00007280  __PyIO_str_newlines
0002:00007290  __PyIO_str_nl
0002:000072a0  __PyIO_str_read
0002:000072b0  __PyIO_str_read1
0002:000072c0  __PyIO_str_readable
0002:000072d0  __PyIO_str_readinto
0002:000072e0  __PyIO_str_readline
0002:000072f0  __PyIO_str_reset
0002:00007300  __PyIO_str_seek
0002:00007310  __PyIO_str_seekable
0002:00007320  __PyIO_str_setstate
0002:00007330  __PyIO_str_tell
0002:00007340  __PyIO_str_truncate
0002:00007350  __PyIO_str_write
0002:00007360  __PyIO_str_writable
0002:00007370  __PyIO_empty_str
0002:00007380  __PyIO_empty_bytes
0002:00007390  __PyIO_zero
0001:0000973d  _PyNumber_AsOff_t
0001:00009850  __PyIO_ConvertSsize_t
0001:00009a57  _init_io
0002:00003ba0  _PyExc_BlockingIOError
0002:000071d8* __PyIO_os_module
0002:000071d0  __PyIO_unsupported_operation
0002:000071d4  __PyIO_locale_module
Module: U:/tmp\ldconv_stringio_obj_18eb52885a17172038.obj(U:\DEV\python-2.7.5\Modules\_io\stringio.c)
0002:00005830  _PyStringIO_Type
Module: U:/tmp\ldconv_textio_obj_18eb52885a171756e8.obj(U:\DEV\python-2.7.5\Modules\_io\textio.c)
0001:0000f38a  __PyIncrementalNewlineDecoder_decode
0001:00010312  __PyIO_find_line_ending
0002:000060f0  _PyIncrementalNewlineDecoder_Type
0002:00006020  _PyTextIOWrapper_Type
0002:000061c0  _PyTextIOBase_Type
Module: U:\usr\local473\lib\libc_dll.lib(dllinit.obj)
0001:00010e60  _DLL_InitTerm
Module: U:\usr\lib\libend.lib(src/libend/386/endlink386.asm)
0002:000073a0  _end
0002:000071c0  _edata
Module: U:\usr\lib\libend.lib(src/libend/386/end.asm)
0001:00010fa0* _etext
0001:00010fa0* __etext
0000:00000000* WEAK$ZERO
0002:000073a0  __end
0002:000071c0  __edata
Module: U:\tmp\ldconv_libgcc_so_d_a_18eb52885a18153fc0.lib(emx-ctordtor.obj)
0001:00010ec0  ___ctordtorInit
0001:00010ef4  ___ctordtorTerm
Module: U:\tmp\ldconv_libgcc_so_d_a_18eb52885a18153fc0.lib(emx-eh.obj)
0001:00010f30  ___ehInit
0001:00010f66* ___ehTerm


                        +----------------------+
                        |   Imported Symbols   |
                        +----------------------+

Symbol                              Module
======                              ======

___libc_ForkRegisterModule          libc065
___init_dll                         libc065
___libc_Back_termDll                libc065
___libc_ForkDeregisterModule        libc065
__atfork_callback                   libc065
_PyErr_SetString                    python27
_PyLong_FromLongLong                python27
_PyLong_FromLong                    python27
_PyObject_CallMethodObjArgs         python27
_PyExc_ValueError                   python27
_PyErr_Occurred                     python27
_PyExc_IOError                      python27
_PyErr_Format                       python27
_PyLong_FromSsize_t                 python27
__PyArg_ParseTuple_SizeT            python27
__PyObject_CallMethod_SizeT         python27
_PyBuffer_Release                   python27
_PyExc_TypeError                    python27
_PyObject_GetAttrString             python27
_PyObject_Repr                      python27
_PyString_FromFormat                python27
_PyExc_AttributeError               python27
_PyErr_ExceptionMatches             python27
_PyErr_Clear                        python27
_PyObject_ClearWeakRefs             python27
_PyMem_Free                         python27
_PyThread_free_lock                 python27
_PyObject_GetAttr                   python27
_PyExc_RuntimeError                 python27
_PyErr_Fetch                        python27
_PyErr_NormalizeException           python27
_PyObject_RichCompareBool           python27
_PyErr_Restore                      python27
_PyBuffer_FillInfo                  python27
_PyMemoryView_FromBuffer            python27
__errno                             libc065
_PyExc_EnvironmentError             python27
__Py_NoneStruct                     python27
_PyNumber_AsSsize_t                 python27
_PyExc_DeprecationWarning           python27
_PyErr_WarnEx                       python27
__Py_TrueStruct                     python27
__PyObject_CallFunction_SizeT       python27
_PyObject_CallObject                python27
__Py_ZeroStruct                     python27
_PyMem_Malloc                       python27
_PyThread_allocate_lock             python27
_PyErr_NoMemory                     python27
__PyArg_ParseTupleAndKeywords_SizeT python27
_PyErr_CheckSignals                 python27
_PyErr_SetObject                    python27
_PyThread_acquire_lock              python27
_PyThread_get_thread_ident          python27
_PyEval_SaveThread                  python27
_PyEval_RestoreThread               python27
_PyThread_release_lock              python27
_PyObject_IsTrue                    python27
_PyString_FromStringAndSize         python27
_PyList_New                         python27
_PyList_Append                      python27
__PyString_Join                     python27
_PyErr_GivenExceptionMatches        python27
__PyString_Resize                   python27
_PyType_GenericNew                  python27
_PyArg_ParseTuple                   python27
_PyExc_OverflowError                python27
_PyNumber_Check                     python27
_PyTuple_Pack                       python27
_PyMem_Realloc                      python27
_PyObject_GetIter                   python27
_PyIter_Next                        python27
_PyObject_GetBuffer                 python27
_PyDict_Copy                        python27
_Py_BuildValue                      python27
_PyDict_Update                      python27
_PyArg_ParseTupleAndKeywords        python27
_PyObject_SelfIter                  python27
_PyUnicodeUCS2_FromString           python27
_PyBool_FromLong                    python27
_PyErr_SetFromErrno                 python27
_PyInt_FromLong                     python27
_PyFloat_Type                       python27
_PyType_IsSubtype                   python27
_PyLong_AsLongLong                  python27
__PyLong_AsInt                      python27
_PyByteArray_Type                   python27
_PyObject_AsCharBuffer              python27
_PyObject_SetAttrString             python27
_PyUnicodeUCS2_FromObject           python27
_Py_FileSystemDefaultEncoding       python27
_PyUnicodeUCS2_AsEncodedString      python27
_PyErr_SetFromErrnoWithFilenameObject python27
_PyExc_OSError                      python27
_PyErr_SetFromErrnoWithFilename     python27
_PyObject_GenericGetAttr            python27
_PyType_GenericAlloc                python27
_PyObject_GC_Del                    python27
_PyByteArray_FromStringAndSize      python27
_PyByteArray_AsString               python27
_PyObject_HasAttrString             python27
_PyObject_Size                      python27
_PyByteArray_Resize                 python27
__PyByteArray_empty_string          python27
_PyLong_AsLong                      python27
__PyInt_AsInt                       python27
_PyNumber_Index                     python27
__PyLong_Sign                       python27
_Py_InitModule4                     python27
_PyImport_ImportModule              python27
_PyModule_AddIntConstant            python27
_PyType_Type                        python27
_PyModule_AddObject                 python27
_PyType_Ready                       python27
_PyString_InternFromString          python27
_PyUnicodeUCS2_FromStringAndSize    python27
_PyUnicodeUCS2_FromUnicode          python27
_PyUnicodeUCS2_Replace              python27
__Py_BuildValue_SizeT               python27
_PyString_FromString                python27
_PyUnicodeUCS2_GetSize              python27
_PyTuple_GetSlice                   python27
__PyArg_Parse_SizeT                 python27
_PyString_AsString                  python27
_PyCodec_IncrementalDecoder         python27
_PyCodec_IncrementalEncoder         python27
__PyCodec_Lookup                    python27
_PyExc_ImportError                  python27
_PyUnicodeUCS2_EncodeUTF32          python27
_PyUnicodeUCS2_EncodeUTF16          python27
_PyUnicodeUCS2_EncodeUTF8           python27
_PyUnicodeUCS2_EncodeLatin1         python27
_PyUnicodeUCS2_EncodeASCII          python27
__PyLong_FromByteArray              python27
_PyNumber_Long                      python27
__PyLong_AsByteArray                python27
_PyUnicodeUCS2_Resize               python27
_PyString_Size                      python27
_PyNumber_Add                       python27
_PyUnicodeUCS2_Join                 python27
_PyUnicodeUCS2_Concat               python27
__CRT_init                          libc065
__CRT_term                          libc065
__std_memcpy                        libc065
__std_memchr                        libc065
__std_memmove                       libc065
__std_memset                        libc065
__std_read                          libc065
__std_fstat                         libc065
__std_lseek                         libc065
__std_isatty                        libc065
__std_write                         libc065
__std_close                         libc065
__std_open                          libc065
__std_strerror                      libc065
__std_ftruncate                     libc065
__std_strchr                        libc065
__std_strcmp                        libc065
___ctordtorInit1                    libc065
___ctordtorTerm1                    libc065
___register_frame_table             gcc473
___deregister_frame                 gcc473


                        +--------------------+
                        |   Libraries Used   |
                        +--------------------+

U:\tmp\ldconv_python2_7_dll_a_18eb52885a17177df8.lib
U:\tmp\ldconv_libgcc_so_d_a_18eb52885a18153fc0.lib
U:\usr\lib\libc_alias.lib
U:\usr\local473\lib\libc_dll.lib
U:\usr\lib\libend.lib


                        +-----------------------+
                        |   Linker Statistics   |
                        +-----------------------+

Stack size:  0000 (0.)
Memory size:  00018340 (99136.)
Link time: 00:00.08
